:100000000C9483000C94A5270C94D0270C94FB2708
:100010000C94AF000C94AF000C94AF000C94AF00A4
:100020000C94AF000C94AF000C94AF000C94AF0094
:100030000C94AF000C94AF000C94AF000C94AF0084
:100040000C94AF000C94AF000C944C290C94AF00AE
:100050000C94B32C0C94E92C0C94AF000C94AF00CE
:100060000C94AF000C94AF000C94AF000C94AF0054
:100070000C94AF000C94AF000C94AF000C94E925E5
:100080000C94AF000C94AF000C94AF000000000182
:100090000200090A00000000040308070000000035
:1000A0000000000000000000000000000102040841
:1000B0001020408001020408102040800102040842
:1000C0001020408001020408102040800202020239
:1000D00002020202040404040404040403030303EC
:1000E00003030303010101010101010100002200DA
:1000F000250028002B0000002100240027002A00F2
:10010000F105711E1D2D2092EC3911241FBECFEF79
:10011000D0E4DEBFCDBF11E0A0E0B1E0EAE4F2E65A
:1001200000E00BBF02C007900D92AA3AB107D9F7C1
:1001300029E3AAEAB1E001C01D92AC3EB207E1F7A3
:1001400010E0C3E8D0E004C02197FE010E945E2FBA
:10015000C038D107C9F70E94A02D0C9423310C940C
:100160000000CF93DF931F92CDB7DEB76983DC0128
:10017000ED91FC910280F381E02D41E050E0BE0161
:100180006F5F7F4F09950F90DF91CF91089508958C
:10019000FC011382128288EE93E0A0E0B0E0848339
:1001A0009583A683B78389E491E09183808380E57A
:1001B000848781E085878AE090E09787868789E059
:1001C00090E0918B808B82E090E0938B828B148AFD
:1001D000158A168A178A118E108E138E128E158E1E
:1001E000148E40E050E0BA01CF010C94772DFC0151
:1001F00077876687518B408B338B228B08950F93C3
:100200001F93CF93DF93EC01062F142F60E08E85B0
:100210000E94522B3C852D8580914039882381F0A6
:100220009FB7F89480914039813081F58DB38093E8
:100230003E394DB380913F39809584238DBB9FBF5C
:100240003CBD2DBD0EBD00000DB407FEFDCF8EB52B
:100250001EBD00000DB407FEFDCF1EB580914039D4
:10026000882351F09FB7F8942091403980913E390E
:10027000213079F48DBB9FBF61E08E850E94522BA7
:10028000812FDF91CF911F910F91089590933E3967
:10029000D7CF8FBFF1CF6F7740E00C94FF0068E1BC
:1002A0000C944B0169E10C944B0169E10E944B01F4
:1002B000682F880F770B880B990B0E94EC2D20E09C
:1002C00030E040E85EE30E949C2E08958F929F925A
:1002D000AF92BF92EF92FF920F931F93CF93DF9352
:1002E0008C016AE10E944B01C82FD0E0C8010E9436
:1002F00055010E94B42D4B017B01F8016489758979
:10030000868997890E94EC2D24ED30E843E45EE471
:100310000E94AF2DBE0187FD12C06D597109F7FE15
:1003200011C0680D791DCB01DF91CF911F910F9105
:10033000FF90EF90BF90AF909F908F900895645A78
:100340007109EDCF072E000C880B990B0E94EC2D44
:1003500020EB32E748E85FE30E949C2E0E94B42D18
:10036000E2CFCF93DF93EC0163E10E944B0190E079
:10037000288D398D821B930BDF91CF910895CF93F8
:10038000DF93EC01E881F9810480F581E02D099586
:10039000892B69F0888D998D0196998F888F60E0FF
:1003A000CE010E944B0190E0DF91CF9108958FEF35
:1003B0009FEFFACF0F931F93CF93DF938C0166E0EB
:1003C0000E944B01D82F67E0C8010E944B01C82F43
:1003D00068E0C8010E944B014C2F50E070E060E0E3
:1003E000762F652F542F44276D2B8A019B01082BF4
:1003F000C901B80120E038E448EE51E00E94792FAD
:1004000003E10E941E30B901CA01DF91CF911F9113
:100410000F9108956DE10E944B0190E034E09595B5
:1004200087953A95E1F78A30910574F4FC01EE0F57
:10043000FF1FE80FF91FE95DFE4F60817181828126
:10044000082E000C990B089560E070E0CB01089530
:100450006CE20C944B01CF93DF93EC0143E861E82D
:100460000E94FF0062E1CE010E944B0183FD03C0A8
:100470000E944B29F7CF48E062E9CE010E94FF00BD
:1004800081E090E0DF91CF910895AF92BF92CF923B
:10049000DF92FF920F931F93CF93DF936C015B0169
:1004A000EA0162E20E944B01F82E90E09C012C0FC1
:1004B0003D1F2F3F310529F020F0CFEFD0E0C81BC2
:1004C000D90B8501AC0EBD1E0A151B0541F0F801C4
:1004D00041918F0160E8C6010E94FF00F5CF4C2FCB
:1004E0004F0D62EAC6010E94FF00CE01DF91CF915D
:1004F0001F910F91FF90DF90CF90BF90AF90089524
:100500000F931F93CF93DF93EC01E881F98104806F
:10051000F581E02D0995892BB1F06DE0CE010E94A7
:100520004B01082F60E0CE010E944B01182F402F95
:100530006DE8CE010E94FF00812F90E0DF91CF9106
:100540001F910F9108958FEF9FEFF8CFCF93DF9317
:10055000EC017D8F6C8F8A899B89672BA1F160E00C
:100560000E94162B40E060ECCE010E94FF008A89B9
:100570009B8982309105D9F08A309105D1F00B9793
:10058000D1F481E00E9425278A899B8982309105D8
:10059000A1F08A30910599F00B9799F481E043E03E
:1005A00050E06DEE75E0DF91CF910C94602782E012
:1005B000E9CF80E0E7CF8FEFE5CF82E0F0CF80E0BA
:1005C000EECF8FEFECCF82309105B9F08A309105F4
:1005D000B1F00B97B1F481E00E948F278A899B8943
:1005E0008230910581F08A30910579F00B9779F48A
:1005F00081E0DF91CF910C94442782E0EDCF80E041
:10060000EBCF8FEFE9CF82E0F4CF80E0F2CF8FEF36
:10061000F0CF41E861E80C94FF0040E861E80C94F9
:10062000FF000E940D030C9411270F931F93CF938B
:10063000DF938C01EB016231710514F0C1E1D0E070
:1006400044E86DECC8010E94FF00C230D10514F4EB
:10065000C2E0D0E0C2504C2F406869E8C801DF9189
:10066000CF911F910F910C94FF000F931F93CF9385
:10067000DF93452BB9F4EB016F30710514F0CEE038
:10068000D0E08C0144E86DEC0E94FF00D7FDC0E093
:100690004C2F406769E8C801DF91CF911F910F91FE
:1006A0000C94FF00DF91CF911F910F910C941503D3
:1006B000AF92BF92CF92DF92EF92FF920F931F9370
:1006C000CF93DF93EC01DB01CA018C8B9D8BAE8B4A
:1006D000BF8B6A017B01FF0CCC08DC2C76019A01F0
:1006E000AB016C2D7C2D8C2D9C2D03E10E940330E1
:1006F000A12CE8E4BE2EF8EECF2EDD24D394E12C1D
:10070000F12C00E010E00E94A62F122FC22ED32E53
:100710007A01A7016627772766E8CE010E94FF00CD
:1007200077276F2D5E2D4D2D67E8CE010E94FF00CB
:10073000412F68E8CE01DF91CF911F910F91FF907B
:10074000EF90DF90CF90BF90AF900C94FF00CF92CE
:10075000DF92EF92FF92CF93DF93EC016A017B016E
:1007600061E08E850E94162B61E08E850E94522BDF
:10077000888999898F3F9807B9F061E00E94162B0C
:1007800060E088890E94522B6AE070E080E090E08F
:100790000E94C72961E088890E94522B6AE070E0BC
:1007A00080E090E00E94C7290E94DB2662E4CE012F
:1007B0000E944B01823191F5CE010E940D03B701D9
:1007C000A601CE010E94580340E06EE8CE010E94CF
:1007D000FF0040E06FE8CE010E94FF006CE0CE0118
:1007E0000E944B01482F43606CE8CE010E94FF003D
:1007F00044E066EACE010E94FF0062E070E0CE01B4
:100800000E941503CE010E94090381E090E0DF9170
:10081000CF91FF90EF90DF90CF90089590E080E02F
:10082000F6CFCF92DF92EF92FF92CF93DF93EC015E
:100830006EE10E944B01F82ECE010E940A02F29452
:100840002FE0F222CC24C394D12C02C0CC0CDD1CAE
:10085000FA94E2F70D2C000CEE08FF0828EE33E0C6
:1008600040E050E00E943F2FC701B6010E943F2F99
:1008700021313105410551055CF04CE066EACE01BD
:10088000DF91CF91FF90EF90DF90CF900C94FF001D
:1008900044E0F4CF0F931F93CF93DF938C01EB01D0
:1008A0006630710534F06D30710534F566307105D0
:1008B00029F545EC61EBC8010E94FF004CE067EBB5
:1008C000C8010E94FF00C6E0D0E06EE1C8010E94AE
:1008D0004B018F7094E0CC0FDD1F9A95E1F74C2F00
:1008E000482B6EE9C8010E94FF00C801DF91CF913B
:1008F0001F910F910C941104CCE0D0E043EC61EB1C
:10090000C8010E94FF004AE067EBC8010E94FF0097
:10091000DCCFCF92DF92EF92FF920F931F93CF9392
:10092000DF938C01CB01BA010E94EC2D6B017C019D
:1009300020E030EC43EF55E40E94AF2DD0E0C0E062
:1009400018160CF065C020E030E842E256E4C7011A
:10095000B6010E94AF2DC1E0D0E018160CF058C0CF
:1009600020E030EC43E756E4C701B6010E94AF2D0A
:10097000C2E0D0E018160CF04BC020E030E842EAAC
:1009800056E4C701B6010E94AF2DC3E0D0E01816AF
:100990000CF03EC020E034E244EF56E4C701B6015B
:1009A0000E94AF2DC4E0D0E0181694F520E034EE9C
:1009B00042E257E4C701B6010E94AF2DC5E0D0E086
:1009C000181634F520E034E244E757E4C701B601D5
:1009D0000E94AF2DC6E0D0E01816D4F420E034E237
:1009E00044EF57E4C701B6010E94AF2DC7E0D0E045
:1009F000181674F420E034E244E758E4C701B60165
:100A00000E94AF2DC9E0D0E0181614F0C8E0D0E085
:100A10006DE1C8010E944B018F7094E0CC0FDD1F87
:100A20009A95E1F74C2F482B6DE9C8010E94FF0011
:100A3000C801DF91CF911F910F91FF90EF90DF9050
:100A4000CF900C9411040F931F93CF93DF938C01DD
:100A5000EB016930710514F0C8E0D0E06DE1C80128
:100A60000E944B01C530D10514F4C5E0D0E02497B5
:100A7000CC0FDD1F482F417F4C2B6DE9C801DF9162
:100A8000CF911F910F910C94FF00CF93DF93EC0156
:100A90006EE10E944B01482F44606EE9CE01DF9168
:100AA000CF910C94FF00CF93DF93EC011B8E1A8E35
:100AB0006DE10E944B01482F4E7F6DE9CE01DF9121
:100AC000CF910C94FF00CF93DF93EC0181E090E095
:100AD0009B8F8A8F6DE1CE010E944B01482F4160B0
:100AE0006DE9CE01DF91CF910C94FF000F931F931E
:100AF000CF93DF93EC018B010E940903CE01012B00
:100B000099F00E94630540E06DE8CE010E94FF006D
:100B100040E062EACE010E94FF0081E090E0DF91B8
:100B2000CF911F910F9108950E945305ECCF0F9321
:100B30001F93CF93DF93EC018B011616170684F4F5
:100B40000E946305402F62EACE010E94FF0045E843
:100B500061E8CE01DF91CF911F910F910C94FF00BE
:100B60000E945305F4CF0F931F93CF93DF93EC01B3
:100B700062E10E944B01182F482F62E9CE010E94CA
:100B8000FF0015FD25C0198E188E8A8D9B8D62E29F
:100B9000892B09F463E1CE010E944B01082F10E07C
:100BA00060E1CE010E944B01482F6DE8CE010E940A
:100BB000FF00EC8DFD8D309711F0C801099540E0E4
:100BC0006DE8CE01DF91CF911F910F910C94FF0042
:100BD000DF91CF911F910F9108958AEA91E00C94D3
:100BE000B3058AEA91E00C94C8002F923F924F928D
:100BF0005F926F927F928F929F92AF92BF92CF92AD
:100C0000DF92EF92FF920F931F93CF93DF93CDB7B5
:100C1000DEB7C857D1090FB6F894DEBF0FBECDBFFF
:100C2000E9969FAF8EAFE9971A01DC0118960D91F6
:100C30001D912D913C911B9761960CAF1DAF2EAF6E
:100C40003FAF61971C960D911D912D913C911F977F
:100C500009831A832B833C8350960D911D912D910E
:100C60003C9153970D831E832F83388754960D91A3
:100C70001D912D913C91579709871A872B873C87A7
:100C8000E6966FAFE697E7967FAFE797A85ABF4F14
:100C90006396BFAFAEAF6397FC01E45AFF4F659612
:100CA000FFAFEEAF65978C01005A1F4F67961FAFDD
:100CB0000EAF67979C012C593F4F69963FAF2EAFFF
:100CC000699788599F4F6B969FAF8EAF6B97E99648
:100CD000AEADBFADE997A459BF4F6D96BFAFAEAFF4
:100CE0006D97E996EEADFFADE997E059FF4F6F962E
:100CF000FFAFEEAF6F97E9960EAD1FADE9970C58B9
:100D00001F4FA1961FAF0EAFA197E9962EAD3FAD35
:100D1000E99728583F4FA3963FAF2EAFA397E99688
:100D20008EAD9FADE99784589F4FA5969FAF8EAF2C
:100D3000A597E996AEADBFADE997A058BF4FA7966E
:100D4000BFAFAEAFA797E996EEADFFADE997EC5711
:100D5000FF4FA996FFAFEEAFA997E9960EAD1FAD75
:100D6000E99708571F4FAB961FAF0EAFAB97E996A9
:100D70002EAD3FADE99724573F4FAD963FAF2EAF15
:100D8000AD97E9968EAD9FADE99780579F4FAF968F
:100D90009FAF8EAFAF97E996AEADBFADE997AC56BA
:100DA000BF4FE196BFAFAEAFE197E796AEADBFAD37
:100DB000E7970D911D912D913C910D871E872F87EF
:100DC000388B6396EEADFFAD63970083118322836A
:100DD000338361968CAD9DADAEADBFAD6197885844
:100DE0009B45A549B842800F911FA21FB31F4D819B
:100DF0005E816F81788509851A852B853C85402722
:100E000051276227732709811A812B813C81402356
:100E100051236223732309851A852B853C8540273E
:100E2000512762277327840F951FA61FB71F8C01B8
:100E30009D0147E0000F111F221F331F4A95D1F774
:100E4000AC01BD01E9E17695679557954795EA951F
:100E5000D1F7402B512B622B732B89819A81AB8167
:100E6000BC81480F591F6A1F7B1FE796AEADBFAD0F
:100E7000E79714960D911D912D913C911797098B31
:100E80001A8B2B8B3C8B6596EEADFFAD659700837F
:100E900011832283338389859A85AB85BC858A5AE1
:100EA0009844A843B741800F911FA21FB31FC98068
:100EB000DA80EB80FC800D811E812F813885C02671
:100EC000D126E226F326C422D522E622F722C02626
:100ED000D126E226F3268C0D9D1DAE1DBF1D8C0173
:100EE0009D01FCE0000F111F221F331FFA95D1F75F
:100EF0006C017D01A4E1F694E794D794C794AA9578
:100F0000D1F7C02AD12AE22AF32AC40ED51EE61E42
:100F1000F71EE796AEADBFADE79718968D919D9100
:100F20000D90BC91A02D8D8B9E8BAF8BB88F67964B
:100F3000EEADFFAD679780839183A283B3838D81EC
:100F40009E81AF81B88585529F48AF4DBB4D0D89BD
:100F50001E892F89388D800F911FA21FB31F4980D2
:100F60005A806B807C8044265526662677264C2046
:100F70005D206E207F2009811A812B813C814026D3
:100F8000512662267326840D951DA61DB71D8C0162
:100F90009D01EFE03695279517950795EA95D1F7CE
:100FA0002C013D01F1E1440C551C661C771CFA959F
:100FB000D1F7402A512A622A732A4C0C5D1C6E1C00
:100FC0007F1CE796AEADBFADE7971C968D919D91C6
:100FD0000D90BC91A02D898F9A8FAB8FBC8F699695
:100FE000EEADFFAD699780839183A283B38389813E
:100FF0009A81AB81BC8182519143A244BE43098D49
:101000001A8D2B8D3C8D800F911FA21FB31F8A015B
:101010009B010C251D252E253F2504211521262168
:1010200037210427152726273727800F911FA21F56
:10103000B31F4C015D011AE0B694A794979487946E
:101040001A95D1F78C019D0186E1000F111F221F17
:10105000331F8A95D1F7082919292A293B29040D1C
:10106000151D261D371DE796AEADBFADE79750960F
:101070008D919D910D90BC91A02D8D8F9E8FAF8FE6
:10108000B8A36B96EEADFFAD6B9780839183A2837F
:10109000B3838155904FA348BA40840F951FA61F74
:1010A000B71FB701A601442555256625772540239E
:1010B0005123622373234C255D256E257F25840FE4
:1010C000951FA61FB71F4C015D0147E0880C991CB6
:1010D000AA1CBB1C4A95D1F7AC01BD01E9E176958C
:1010E000679557954795EA95D1F7482959296A296F
:1010F0007B29400F511F621F731FE796AEADBFAD36
:10110000E79754968D919D910D90BC91A02D89A348
:101110009AA3ABA3BCA36D96EEADFFAD6D97808394
:101120009183A283B383865D9943A847B84B8C0D06
:101130009D1DAE1DBF1D73016201C026D126E22692
:10114000F326C422D522E622F722C424D524E6249D
:10115000F7248C0D9D1DAE1DBF1D4C015D01FCE0F3
:10116000880C991CAA1CBB1CFA95D1F76C017D0157
:10117000A4E1F694E794D794C794AA95D1F7C82828
:10118000D928EA28FB28C40ED51EE61EF71EE796CE
:10119000AEADBFADE79758968D919D910D90BC91E6
:1011A000A02D8DA39EA3AFA3B8A76F96EEADFFAD04
:1011B0006F9780839183A283B3838D5E994BAF4CED
:1011C000B745840D951DA61DB71D2801390144267C
:1011D0005526662677264C205D206E207F204026EF
:1011E000512662267326840D951DA61DB71D4C0140
:1011F0005D01EFE0B694A79497948794EA95D1F7B0
:101200002C013D01F1E1440C551C661C771CFA953C
:10121000D1F7482859286A287B284C0C5D1C6E1C85
:101220007F1CE796AEADBFADE7975C968D919D9123
:101230000D90BC91A02D89A79AA7ABA7BCA7A1969A
:10124000EEADFFADA19780839183A283B3838F5FBF
:101250009A46A94BB240800F911FA21FB31F8A016B
:101260009B010C251D252E253F2504211521262116
:1012700037210427152726273727800F911FA21F04
:10128000B31F4C015D011AE0B694A794979487941C
:101290001A95D1F78C019D0186E1000F111F221FC5
:1012A000331F8A95D1F7082919292A293B29040DCA
:1012B000151D261D371DE796AEADBFADE79790967D
:1012C0008D919D910D90BC91A02D8DA79EA7AFA74C
:1012D000B8ABA396EEADFFADA39780839183A283B5
:1012E000B38388529746AF47B649840F951FA61F10
:1012F000B71FB701A601442555256625772540234C
:101300005123622373234C255D256E257F25840F91
:10131000951FA61FB71F4C015D0147E0880C991C63
:10132000AA1CBB1C4A95D1F7AC01BD01E9E1769539
:10133000679557954795EA95D1F7482959296A291C
:101340007B29400F511F621F731FE796AEADBFADE3
:10135000E79794968D919D910D90BC91A02D89ABAE
:101360009AABABABBCABA596EEADFFADA5978083BA
:101370009183A283B38381559840AB4BB4478C0DC6
:101380009D1DAE1DBF1D73016201C026D126E22640
:10139000F326C422D522E622F722C424D524E6244B
:1013A000F7248C0D9D1DAE1DBF1D4C015D01FCE0A1
:1013B000880C991CAA1CBB1CFA95D1F76C017D0105
:1013C000A4E1F694E794D794C794AA95D1F7C828D6
:1013D000D928EA28FB28C40ED51EE61EF71EE7967C
:1013E000AEADBFADE79798968D919D910D90BC9154
:1013F000A02D8DAB9EABAFABB8AFA796EEADFFAD5A
:10140000A79780839183A283B3838F54944AA109C1
:10141000B109840D951DA61DB71D2801390144266B
:101420005526662677264C205D206E207F2040269C
:10143000512662267326840D951DA61DB71D4C01ED
:101440005D01EFE0B694A79497948794EA95D1F75D
:101450002C013D01F1E1440C551C661C771CFA95EA
:10146000D1F7482859286A287B284C0C5D1C6E1C33
:101470007F1CE796AEADBFADE7979C968D919D9191
:101480000D90BC91A02D89AF9AAFABAFBCAFA99620
:10149000EEADFFADA99780839183A283B38382547D
:1014A0009842A34AB647800F911FA21FB31F8A011B
:1014B0009B010C251D252E253F25042115212621C4
:1014C00037210427152726273727800F911FA21FB2
:1014D000B31F4C015D011AE0B694A79497948794CA
:1014E0001A95D1F78C019D0186E1000F111F221F73
:1014F000331F8A95D1F7082919292A293B29040D78
:10150000151D261D371DE796AEADBFADE797D096EA
:101510008D919D910D90BC91A02D21968CAF9DAF8A
:10152000AEAFBFAF2197AB96EEADFFADAB9780836B
:101530009183A283B3834C015D01FEED8F1AFEEE11
:101540009F0AFFE6AF0AF4E9BF0A840E951EA61EA5
:10155000B71EB701A60144255525662577254023EA
:101560005123622373234C255D256E257F25480D6D
:10157000591D6A1D7B1D4A015B0197E0880C991C6F
:10158000AA1CBB1C9A95D1F7E9E17695679557950A
:101590004795EA95D1F7482959296A297B29400FAF
:1015A000511F621F731FE796AEADBFADE797D4968C
:1015B0008D919D910D90BC91A02D25968CAF9DAFE6
:1015C000AEAFBFAF2597AD96EEADFFADAD978083C3
:1015D0009183A283B3834C015D01FDE68F1AFEE87F
:1015E0009F0AF7E6AF0AF2E0BF0A8C0C9D1CAE1C06
:1015F000BF1C73016201C026D126E226F326C42255
:10160000D522E622F722C424D524E624F724C80CE8
:10161000D91CEA1CFB1C46015701FCE0880C991CF4
:10162000AA1CBB1CFA95D1F7A4E1F694E794D794D1
:10163000C794AA95D1F7C828D928EA28FB28C40E50
:10164000D51EE61EF71EE796AEADBFADE797D8965E
:101650008D919D910D90BC91A02D29968CAF9DAF41
:10166000AEAFBFAF2997AF96EEADFFADAF9780831A
:101670009183A283B3834C015D01F2E78F1AFCEBE7
:101680009F0AF6E8AF0AF9E5BF0A840C951CA61C70
:10169000B71C2801390144265526662677264C209A
:1016A0005D206E207F204026512662267326480C3E
:1016B000591C6A1C7B1C53014201BFE0B694A794DD
:1016C00097948794BA95D1F781E1440C551C661C18
:1016D000771C8A95D1F7482859286A287B284C0C12
:1016E0005D1C6E1C7F1CE796AEADBFADE797DC9628
:1016F0008D919D910D90BC91A02D2D968CAF9DAF9D
:10170000AEAFBFAF2D97E196EEADFFADE197808311
:101710009183A283B3834C015D01FFED8F1AF7EF34
:101720009F0AFBE4AF0AF6EBBF0A800E911EA21ED1
:10173000B31E8A019B010C251D252E253F25042162
:101740001521262137210427152726273727080D9D
:10175000191D2A1D3B1D480159019AE0B694A79412
:10176000979487949A95D1F7E6E1000F111F221FF5
:10177000331FEA95D1F7082919292A293B29040D95
:10178000151D261D371D89889A88AB88BC888EE96F
:10179000881A8AED980A81EEA80A89E0B80A840EB0
:1017A000951EA61EB71EB301A2014027512762272E
:1017B00073274C215D216E217F2144255525662507
:1017C0007725480D591D6A1D7B1D4A015B01F5E017
:1017D000880C991CAA1CBB1CFA95D1F7ABE1769535
:1017E000679557954795AA95D1F7482959296A29A8
:1017F0007B29400F511F621F731F8DA09EA0AFA0B9
:10180000B8A490EC891A9CE4990A9FEBA90A9FE37B
:10181000B90A8C0C9D1CAE1CBF1C68017901C42642
:10182000D526E626F726C420D520E620F720C026B8
:10183000D126E226F326C80CD91CEA1CFB1C460163
:101840005701B9E0880C991CAA1CBB1CBA95D1F7AA
:1018500087E1F694E794D794C7948A95D1F7C8287E
:10186000D928EA28FB28C40ED51EE61EF71E89AC2F
:101870009AACABACBCACAFEA8A1AA5EA9A0AA1EA68
:10188000AA0AA9EDBA0A840C951CA61CB71C2A0149
:101890003B014C245D246E247F244022512262228D
:1018A00073224426552666267726480C591C6A1C46
:1018B0007B1C530142019EE0880C991CAA1CBB1C96
:1018C0009A95D1F7E2E17694679457944794EA9514
:1018D000D1F7482859286A287B284C0C5D1C6E1CBF
:1018E0007F1C8D849E84AF84B888B6E58B1AB8E3DC
:1018F0009B0AB9E4AB0AB6E1BB0A800E911EA21E98
:10190000B31E9701860104251525262537250423B6
:101910001523262337230C251D252E253F25080DAD
:10192000191D2A1D3B1D48015901FCE0B694A794DE
:1019300097948794FA95D1F7A4E1000F111F221F05
:10194000331FAA95D1F7082919292A293B29040D03
:10195000151D261D371D89A09AA0ABA0BCA0E3EAE7
:101960008E1AEFEE9E0AE0EDAE0AE9E2BE0A840EA0
:10197000951EA61EB71EB301A2014027512762275C
:1019800073274C215D216E217F2144255525662535
:101990007725480D591D6A1D7B1D4A015B01B5E085
:1019A000880C991CAA1CBB1CBA95D1F78BE17695C3
:1019B0006795579547958A95D1F7482959296A29F6
:1019C0007B29400F511F621F731F8DA89EA8AFA8CF
:1019D000B8ACFDEA8F1AFBEE9F0AFBEBAF0AFDEFF6
:1019E000BF0A8C0C9D1CAE1CBF1C68017901C4266B
:1019F000D526E626F726C420D520E620F720C026E7
:101A0000D126E226F326C80CD91CEA1CFB1C460191
:101A1000570199E0880C991CAA1CBB1C9A95D1F718
:101A2000E7E1F694E794D794C794EA95D1F7C828EC
:101A3000D928EA28FB28C40ED51EE61EF71E2D96CF
:101A40008CAC9DACAEACBFAC2D978FE7881A89E10A
:101A5000980A8EE5A80A87E2B80A840C951CA61C91
:101A6000B71C2A013B014C245D246E247F244022B4
:101A70005122622273224426552666267726480C78
:101A8000591C6A1C7B1C53014201FEE0880C991C06
:101A9000AA1CBB1CFA95D1F7A2E1769467945794DF
:101AA0004794AA95D1F7482859286A287B284C0CD6
:101AB0005D1C6E1C7F1C8D8C9E8CAF8CB8A098E337
:101AC000891A94E0990A9CE2A90A98E1B90A800E61
:101AD000911EA21EB31E97018601042515252625F9
:101AE000372504231523262337230C251D252E25D2
:101AF0003F25080D191D2A1D3B1D48015901BCE059
:101B0000B694A79497948794BA95D1F784E1000F7F
:101B1000111F221F331F8A95D1F7082919292A2955
:101B20003B29040D151D261D371D89A89AA8ABA8B1
:101B3000BCA8AAE18A1AA2E39A0AAEE1AA0AAEED0B
:101B4000BA0A840E951EA61EB71EB301A201402735
:101B50005127622773274C215D216E217F21442567
:101B6000552566257725480D591D6A1D7B1D4A019F
:101B70005B0195E0880C991CAA1CBB1C9A95D1F7B7
:101B8000EBE17695679557954795EA95D1F7482902
:101B900059296A297B29400F511F621F731F2996FB
:101BA0008CAC9DACAEACBFAC2997BAE28B1AB8EF47
:101BB0009B0AB8ECAB0ABCE3BB0A8C0C9D1CAE1CA8
:101BC000BF1C68017901C426D526E626F726C42065
:101BD000D520E620F720C026D126E226F326C80C21
:101BE000D91CEA1CFB1C46015701F9E0880C991C22
:101BF000AA1CBB1CFA95D1F7A7E1F694E794D794F9
:101C0000C794AA95D1F7C828D928EA28FB28C40E7A
:101C1000D51EE61EF71E898C9A8CAB8CBC8CE9E72E
:101C20008E1AE2EF9E0AEAE2AE0AEBE0BE0A840CEC
:101C3000951CA61CB71C2A013B014C245D246E2474
:101C40007F24402251226222732244265526662692
:101C50007726480C591C6A1C7B1C53014201BEE0CC
:101C6000880C991CAA1CBB1CBA95D1F782E176940A
:101C70006794579447948A95D1F7482859286A2839
:101C80007B284C0C5D1C6E1C7F1C8DA49EA4AFA4F5
:101C9000B8A8F3E18F1AFBEE9F0AF5EAAF0AFAEB58
:101CA000BF0A800E911EA21EB31E97018601042555
:101CB00015252625372504231523262337230C2510
:101CC0001D252E253F25080D191D2A1D3B1D4801E8
:101CD00059019CE0B694A794979487949A95D1F76C
:101CE000E4E1000F111F221F331FEA95D1F70829E5
:101CF00019292A293B29040D151D261D371D259656
:101D00008CAC9DACAEACBFAC25978BEF881A86E14E
:101D1000980A8CE1A80A86E5B80A840E951EA61ECC
:101D2000B71EB301A20140275127622773274C2118
:101D30005D216E217F214425552566257725480D97
:101D4000591D6A1D7B1D4A015B01F5E0880C991C39
:101D5000AA1CBB1CFA95D1F7ABE176956795579510
:101D60004795AA95D1F7482959296A297B29400F17
:101D7000511F621F731F8D889E88AF88B88C98E0B2
:101D8000891A9CE5990A90E1A90A93E0B90A8C0C9A
:101D90009D1CAE1CBF1C68017901C426D526E62611
:101DA000F726C420D520E620F720C026D126E2263B
:101DB000F326C80CD91CEA1CFB1C46015701B9E0EC
:101DC000880C991CAA1CBB1CBA95D1F787E1F69424
:101DD000E794D794C7948A95D1F7C828D928EA28D8
:101DE000FB28C40ED51EE61EF71E89A49AA4ABA438
:101DF000BCA4A7E28A1AADEF9A0AA0E9AA0AA8E948
:101E0000BA0A840C951CA61CB71C2A013B014C2461
:101E10005D246E247F2440225122622273224426B4
:101E2000552666267726480C591C6A1C7B1C5301D4
:101E300042019EE0880C991CAA1CBB1C9A95D1F704
:101E4000E2E17694679457944794EA95D1F748284D
:101E500059286A287B284C0C5D1C6E1C7F1C46018F
:101E6000570184249524A624B72421968CAD9DADDA
:101E7000AEADBFAD21978657934BA54DB247800FAE
:101E8000911FA21FB31F950184010423152326234C
:101E900037230C251D252E253F25800F911FA21FBE
:101EA000B31F8C019D01FCE036952795179507958A
:101EB000FA95D1F7E5960CAF1DAF2EAF3FAFE59782
:101EC0008C019D01A4E1000F111F221F331FAA9551
:101ED000D1F7E5968CAD9DADAEADBFADE597082BC6
:101EE000192B2A2B3B2B040D151D261D371D89A1EF
:101EF0009AA1ABA1BCA18E5B964CA540B109840F01
:101F0000951FA61FB71F80269126A226B326880EEE
:101F1000991EAA1EBB1ED501C40144E0880F991F5B
:101F2000AA1FBB1F4A95D1F75CE1B694A79497947A
:101F300087945A95D1F7882A992AAA2ABB2A800E13
:101F4000911EA21EB31E4DA55EA56FA578A94F5781
:101F500059406E4878474C0D5D1D6E1D7F1D730105
:101F60006201C026D126E226F326C824D924EA2419
:101F7000FB24C40ED51EE61EF71EB701A601EBE03A
:101F8000440F551F661F771FEA95D1F7F5E1F694C8
:101F9000E794D794C794FA95D1F7C42AD52AE62AAC
:101FA000F72AC80CD91CEA1CFB1C49AD5AAD6BAD15
:101FB0007CAD4E5D5E4962467249440E551E661EFA
:101FC000771EB901A801482559256A257B254C258E
:101FD0005D256E257F25440E551E661E771ED20197
:101FE00023013D014C0C5D1C6E1C7F1C29964CADE1
:101FF0005DAD6EAD7FAD2997445F574C6A4172402D
:10200000400F511F621F731F950184010C251D2570
:102010002E253F250425152526253725040F151FB8
:10202000261F371FB901A801A9E076956795579536
:102030004795AA95D1F7B7E1000F111F221F331F53
:10204000BA95D1F7042B152B262B372B040D151D14
:10205000261D371D49895A896B897C894C5B5541FE
:1020600061447B45480D591D6A1D7B1D4601570182
:1020700084249524A624B72480269126A226B3265C
:10208000840E951EA61EB71EB501A40184E0440F60
:10209000551F661F771F8A95D1F79CE1B694A794C8
:1020A000979487949A95D1F7842A952AA62AB72AD5
:1020B000800E911EA21EB31E4D8D5E8D6F8D78A178
:1020C000475550436142744BC40ED51EE61EF71EA1
:1020D000B301A201402751276227732748255925BC
:1020E0006A257B254C0D5D1D6E1D7F1DDB01CA0120
:1020F000EBE0880F991FAA1FBB1FEA95D1F7F5E106
:102100007695679557954795FA95D1F7482B592BB2
:102110006A2B7B2B480D591D6A1D7B1DC9A4DAA4AF
:10212000EBA4FCA4B0EACB1AB4EBDB0AB4E4EB0AF0
:10213000B9E0FB0A4C0C5D1C6E1C7F1C6801790128
:10214000C824D924EA24FB24C426D526E626F7266B
:102150004C0C5D1C6E1C7F1CF20123013F01440EE0
:10216000551E661E771ECDA8DEA8EFA8F8ACF0E9D4
:10217000CF1AF3E4DF0AF0E4EF0AF1E4FF0AC00E3D
:10218000D11EE21EF31E9501840104271527262780
:10219000372704251525262537250C0D1D1D2E1D39
:1021A0003F1D68017901A9E0F694E794D794C7949C
:1021B000AA95D1F7B7E1000F111F221F331FBA955F
:1021C000D1F70C291D292E293F29040D151D261D87
:1021D000371D2596CCACDDACEEACFFAC25978AE381
:1021E000C81A81E8D80A84E6E80A87EDF80AC80C1C
:1021F000D91CEA1CFB1C4A015B0184249524A624FB
:10220000B72480269126A226B3268C0C9D1CAE1CDA
:10221000BF1C7501640184E0CC0CDD1CEE1CFF1CAE
:102220008A95D1F79CE1B694A794979487949A9550
:10223000D1F78C289D28AE28BF28800E911EA21EA3
:10224000B31ECD84DE84EF84F88896E0C91A98ED39
:10225000D90A9EE5E90A95E1F90AC40ED51EE61EE3
:10226000F71EB301A2014027512762277327482593
:1022700059256A257B254C0D5D1D6E1D7F1D6A014C
:102280007B01EBE0CC0CDD1CEE1CFF1CEA95D1F7CA
:10229000F5E17695679557954795FA95D1F74C29CD
:1022A0005D296E297F29480D591D6A1D7B1DC98C2A
:1022B000DA8CEB8CFC8CABE7CA1AAFECDA0AA0E143
:1022C000EA0AABE2FA0A4C0C5D1C6E1C7F1C68012A
:1022D0007901C824D924EA24FB24C426D526E6267D
:1022E000F7264C0C5D1C6E1C7F1CF20123013F0184
:1022F000440E551E661E771ECDA0DEA0EFA0F8A4EA
:10230000FBEFCF1AF2EEDF0AF7E7EF0AFBEFFF0A67
:10231000C00ED11EE21EF31E95018401042715276D
:102320002627372704251525262537250C0D1D1DA5
:102330002E1D3F1D68017901A9E0F694E794D7941A
:10234000C794AA95D1F7B7E1000F111F221F331FC1
:10235000BA95D1F70C291D292E293F29040D151DE9
:10236000261D371DC9A8DAA8EBA8FCA887ECC81A57
:102370008FE2D80A8BE2E80A86E2F80AC80CD91C78
:10238000EA1CFB1C4A015B0184249524A624B72483
:1023900080269126A226B3268C0C9D1CAE1CBF1C49
:1023A0007501640184E0CC0CDD1CEE1CFF1C8A95D9
:1023B000D1F79CE1B694A794979487949A95D1F716
:1023C0008C289D28AE28BF28800E911EA21EB31E09
:1023D0002196CCACDDACEEACFFAC21979BE1C91AE9
:1023E00096E6D90A94E2E90A99E1F90AC40ED51EE3
:1023F000E61EF71EB301A20140275127622773276B
:10240000482559256A257B254C0D5D1D6E1D7F1DB8
:102410006A017B01EBE0CC0CDD1CEE1CFF1CEA9595
:10242000D1F7F5E17695679557954795FA95D1F7E8
:102430004C295D296E297F29480D591D6A1D7B1D78
:102440002D96CCACDDACEEACFFAC2D97A8E0CA1A53
:10245000A3E8DA0AADE5EA0AA0EEFA0A4C0C5D1C24
:102460006E1C7F1C68017901C824D924EA24FB244E
:10247000C426D526E626F7264C0C5D1C6E1C7F1C58
:10248000F20123013F01440E551E661E771ECD88C2
:10249000DE88EF88F88CFBE9CF1AF9EADF0AF3E56A
:1024A000EF0AFBE3FF0AC00ED11EE21EF31E9501E8
:1024B00084010427152726273727042515252625D7
:1024C00037250C0D1D1D2E1D3F1D68017901A9E04A
:1024D000F694E794D794C794AA95D1F7B7E1000F83
:1024E000111F221F331FBA95D1F70C291D292E2940
:1024F0003F29040D151D261D371DCD84DE84EF8474
:10250000F8888CEBC81A8DEDD80A86EDE80A8BE0C6
:10251000F80AC80CD91CEA1CFB1C4A015B01809418
:102520009094A094B094802A912AA22AB32A842459
:102530009524A624B7248C0C9D1CAE1CBF1C7501D1
:10254000640186E0CC0CDD1CEE1CFF1C8A95D1F7E3
:102550009AE1B694A794979487949A95D1F78C288A
:102560009D28AE28BF28800E911EA21EB31EC9A4AE
:10257000DAA4EBA4FCA499E6C91AD10895EDE90AFE
:102580009CEBF90AC40ED51EE61EF71EB301A2018C
:102590004095509560957095482959296A297B295D
:1025A00040275127622773274C0D5D1D6E1D7F1D2F
:1025B0006A017B01EAE0CC0CDD1CEE1CFF1CEA95F5
:1025C000D1F7F6E17695679557954795FA95D1F746
:1025D0004C295D296E297F29480D591D6A1D7B1DD7
:1025E0002996CCACDDACEEACFFAC2997A9E5CA1AB4
:1025F000ACEDDA0AABE6EA0AA4E5FA0AC40CD51C8B
:10260000E61CF71C280139014094509460947094A2
:10261000442A552A662A772A482459246A247B2486
:102620004C0C5D1C6E1C7F1C73016201AFE0CC0C76
:10263000DD1CEE1CFF1CAA95D1F7B1E176946794DE
:1026400057944794BA95D1F74C285D286E287F2877
:10265000440E551E661E771EC9A0DAA0EBA0FCA092
:10266000B7ECCB1ABFE5DB0ABCE6EB0AB3E0FB0A2A
:10267000C00ED11EE21EF31E950184010095109537
:10268000209530950429152926293729042715274F
:10269000262737270C0D1D1D2E1D3F1D68017901B2
:1026A0008BE0F694E794D794C7948A95D1F795E197
:1026B000000F111F221F331F9A95D1F70C291D29D6
:1026C0002E293F29040D151D261D371D2196CCAC42
:1026D000DDACEEACFFAC2197EDE3CE1AE6EADE0A04
:1026E000E4EAEE0AEAE9FE0AC80CD91CEA1CFB1C63
:1026F0004A015B0180949094A094B094802A912A1E
:10270000A22AB32A84249524A624B7248C0C9D1CC9
:10271000AE1CBF1C75016401E6E0CC0CDD1CEE1C98
:10272000FF1CEA95D1F7FAE1B694A79497948794A1
:10273000FA95D1F78C289D28AE28BF28800E911ECF
:10274000A21EB31EC98CDA8CEB8CFC8CFEE6CF1A71
:10275000F3E3DF0AF3EFEF0AF0E7FF0AC40ED51E3A
:10276000E61EF71EB301A201409550956095709545
:10277000482959296A297B2940275127622773272D
:102780004C0D5D1D6E1D7F1D6A017B01AAE0CC0C06
:10279000DD1CEE1CFF1CAA95D1F7B6E17695679576
:1027A00057954795BA95D1F74C295D296E297F2910
:1027B000480D591D6A1D7B1DCDA8DEA8EFA8F8ACF9
:1027C00083E8C81A8BE0D80A80E1E80AF108C40C53
:1027D000D51CE61CF71C28013901409450946094E4
:1027E0007094442A552A662A772A482459246A2450
:1027F0007B244C0C5D1C6E1C7F1C730162018FE0FE
:10280000CC0CDD1CEE1CFF1C8A95D1F791E176946F
:102810006794579447949A95D1F74C285D286E2871
:102820007F28440E551E661E771EC988DA88EB88FD
:10283000FC889FE2C91A92EAD90A9BE7E90A9AE75B
:10284000F90AC00ED11EE21EF31E95018401009507
:102850001095209530950429152926293729042714
:102860001527262737270C0D1D1D2E1D3F1D68011E
:102870007901EBE0F694E794D794C794EA95D1F701
:10288000F5E1000F111F221F331FFA95D1F70C2914
:102890001D292E293F29040D151D261D371DCDA4E8
:1028A000DEA4EFA4F8A8A1EBCA1AA1E8DA0AA7E50A
:1028B000EA0AA0E9FA0AC80CD91CEA1CFB1C4A0166
:1028C0005B0180949094A094B094802A912AA22ACB
:1028D000B32A84249524A624B7248C0C9D1CAE1CFA
:1028E000BF1C75016401A6E0CC0CDD1CEE1CFF1CB6
:1028F000AA95D1F7BAE1B694A79497948794BA951C
:10290000D1F78C289D28AE28BF28800E911EA21ECC
:10291000B31E2D968CAD9DADAEADBFAD2D97805243
:102920009941A34DB140840F951FA61FB71FB30156
:10293000A2014095509560957095482959296A29BA
:102940007B294027512762277327840F951FA61FD5
:10295000B71F6C017D014AE0CC0CDD1CEE1CFF1C96
:102960004A95D1F7AC01BD01E6E17695679557959B
:102970004795EA95D1F74C295D296E297F29480DA5
:10298000591D6A1D7B1D8DA19EA1AFA1B8A58C5EAE
:102990009C4BAE4FBC45840D951DA61DB71D28014F
:1029A00039014094509460947094442A552A662AC0
:1029B000772A482459246A247B24840D951DA61D5A
:1029C000B71D6C017D01FFE0CC0CDD1CEE1CFF1C73
:1029D000FA95D1F72C013D01A1E1769467945794C3
:1029E0004794AA95D1F74C285D286E287F28440E7D
:1029F000551E661E771E25968CAD9DADAEADBFAD46
:102A000025978F559E4EA74FB14B800F911FA21F48
:102A1000B31F9501840100951095209530950429E8
:102A20001529262937290427152726273727800F18
:102A3000911FA21FB31F6C017D011BE0F694E79468
:102A4000D794C7941A95D1F78C019D0185E1000FA9
:102A5000111F221F331F8A95D1F70C291D292E29FA
:102A60003F29040D151D261D371D8D8D9E8DAF8DA3
:102A7000B8A18E579148AC4AB840880D991DAA1D3F
:102A8000BB1D4A015B0180949094A094B094802A6D
:102A9000912AA22AB32A84249524A624B724880D37
:102AA000991DAA1DBB1D6C017D01E6E0CC0CDD1C4F
:102AB000EE1CFF1CEA95D1F74C015D01FAE1B694DA
:102AC000A79497948794FA95D1F78C289D28AE28DF
:102AD000BF28800E911EA21EB31E89AD9AADABAD6C
:102AE000BCAD8B5C9D40A54CB244840F951FA61FC6
:102AF000B71FB301A2014095509560957095482984
:102B000059296A297B294027512762277327840F77
:102B1000951FA61FB71F6C017D014AE0CC0CDD1C80
:102B2000EE1CFF1C4A95D1F7AC01BD01E6E176959C
:102B3000679557954795EA95D1F74C295D296E29F8
:102B40007F29480D591D6A1D7B1D8D899E89AF897E
:102B5000B88D85549D42A842B54D840D951DA61D86
:102B6000B71D280139014094509460947094442A10
:102B7000552A662A772A482459246A247B24840DFE
:102B8000951DA61DB71D6C017D01FFE0CC0CDD1C61
:102B9000EE1CFF1CFA95D1F72C013D01A1E17694C2
:102BA000679457944794AA95D1F74C285D286E28CE
:102BB0007F28440E551E661E771E89A99AA9ABA9C7
:102BC000BCA98F569C42A947B441800F911FA21FF8
:102BD000B31F950184010095109520953095042927
:102BE0001529262937290427152726273727800F57
:102BF000911FA21FB31F6C017D011BE0F694E794A7
:102C0000D794C7941A95D1F78C019D0185E1000FE7
:102C1000111F221F331F8A95D1F70C291D292E2938
:102C20003F29040D151D261D371D61968CAD9DADE8
:102C3000AEADBFAD6197880D991DAA1DBB1D6196F4
:102C40008CAF9DAFAEAFBFAF619789819A81AB81E9
:102C5000BC81800F911FA21FB31F89839A83AB830E
:102C6000BC830D811E812F813885040D151D261D05
:102C7000371D0D831E832F83388789859A85AB8501
:102C8000BC85840F951FA61FB71F89879A87AB87BE
:102C9000BC87E796AEADBFADE797A05CBF4FE796A8
:102CA000BFAFAEAFE797B0E42B1A310811F00C9428
:102CB000D50661960CAD1DAD2EAD3FAD6197E99681
:102CC000AEADBFADE99718960D931D932D933C9330
:102CD0001B9709811A812B813C811C960D931D93B2
:102CE0002D933C931F970D811E812F81388550961F
:102CF0000D931D932D933C93539709851A852B852E
:102D00003C8554960D931D932D933C935797E796CE
:102D10008EAD9FADE797C858DF4F0FB6F894DEBF72
:102D20000FBECDBFDF91CF911F910F91FF90EF901C
:102D3000DF90CF90BF90AF909F908F907F906F90DB
:102D40005F904F903F902F900895CF93DF93FC01B9
:102D500081E093E2A5E4B7E680879187A287B387F5
:102D600089E89BEAADECBFEE84879587A687B78795
:102D70008EEF9CEDAAEBB8E9808B918BA28BB38B85
:102D800086E794E5A2E3B0E1848B958BA68BB78BA5
:102D90001082118212821382148215821682178287
:102DA000DF01A85ABF4F80E4ED01982F19929A9540
:102DB000E9F77896DF011D928A95E9F7DF91CF91C7
:102DC00008958F929F92AF92BF92EF92FF920F93CE
:102DD0001F93CF93DF93EC017B018A018881998156
:102DE000AA81BB8170E060E04A015B01880E991EF8
:102DF000AA1EBB1E2FE1B22288829982AA82BB82C0
:102E000088169906AA06BB0668F48C809D80AE8061
:102E1000BF802FEF821A920AA20AB20A8C829D8288
:102E2000AE82BF828F739927AA27BB270097A1057F
:102E3000B10579F120E4822E912CA12CB12C881AB5
:102E4000990AAA0ABB0A48968C0F9D1F4815590576
:102E50006A057B0570F4A801B701DF91CF911F913E
:102E60000F91FF90EF90BF90AF909F908F900C9438
:102E7000F530A401B7010E94F530E80CF91C0819DF
:102E8000190940E450E0BE01685E7F4FCE010E9408
:102E9000F5050034110548F0A801407CB701CE01CA
:102EA0000E94F5057C010F731127A801B701CE011F
:102EB0004896D3CFEF92FF920F931F93CF93DF9358
:102EC0008C01EB01488159816A817B814F735527C1
:102ED00066277727DB01CA010196A11DB11D4C0FA2
:102EE0005D1F20E8FA01208F40E450E060E070E0D0
:102EF000481B590B6A0B7B0B7E01F8E1EF0EF11CAE
:102F00004830510561057105A0F4489670E060E015
:102F10008C0F9D1F0E94FE3040E450E0B701CE01AF
:102F20000E94F50540E450E060E070E080E090E051
:102F3000DC0148505109489670E060E08C0F9D1FFD
:102F40000E94FE3088819981AA81BB8123E0880F8D
:102F5000991FAA1FBB1F2A95D1F788839983AA833B
:102F6000BB83FE01E05BFF4F8083319690833196F7
:102F7000A0833196B0833C812D819E818F813196D3
:102F8000308331962083319690833196808340E45C
:102F900050E0B701CE010E94F5058885F8018083D5
:102FA000898581838A8582838B8583838C858483CD
:102FB0008D8585838E8586838F85878388898087A5
:102FC000898981878A8982878B8983878C8984878D
:102FD0008D8985878E8986878F89878788E9FE0115
:102FE00011928A95E9F7DF91CF911F910F91FF9090
:102FF000EF900895CF92DF92EF92FF920F931F937D
:10300000CF93DF93CDB7DEB7C859D1090FB6F89487
:10301000DEBF0FBECDBF7C016B0180E190E00E945E
:1030200026288C01CE0101960E94A516A601B701A3
:10303000CE0101960E94E116BE016F5F7F4FC8016D
:103040000E945A17C801C856DF4F0FB6F894DEBF6A
:103050000FBECDBFDF91CF911F910F91FF90EF90E9
:10306000DF90CF9008951F93CF93DF93EC01162F3D
:103070000E940531181739F0612FCE01DF91CF91F1
:103080001F910C940D31DF91CF911F9108950C94F5
:103090000531DC01ED91FC910190F081E02D099466
:1030A00061E08CE00C94522B60E08CE00C94522B8D
:1030B00061E08DE00C94522B60E08DE00C94522B7B
:1030C00088E198E00FB6F894A895809360000FBE51
:1030D000909360000E9458180E945418FBCF0F93E1
:1030E0001F93CF93DF938C01EC01892B11F4C1E086
:1030F000D0E01C161D060CF561E08CE00E94522BFE
:1031000060E08DE00E94522B64E670E080E090E089
:103110000E94C72960E08CE00E94522B61E08DE0A4
:103120000E94522B64E670E080E090E00E94C72984
:1031300001151105F1F22197DCCF0E945418DF919F
:10314000CF911F910F910C945C180E9458180E9407
:1031500054186AE070E080E090E00E94C7290E9465
:1031600050180E945C1865E070E080E090E00E94DA
:10317000C729EBCF0F931F93CF93DF938C01EC0103
:10318000892B11F4C1E0D0E061E08DE00E94522B68
:103190001C161D06ACF40E945C1864E670E080E02A
:1031A00090E00E94C7290E94581864E670E080E011
:1031B00090E00E94C7290115110551F32197E8CF2E
:1031C000DF91CF911F910F910C945C180F931F9377
:1031D000CF93DF938C01EC01892B11F4C1E0D0E097
:1031E0001C161D06ACF40E94541864E670E080E0E2
:1031F00090E00E94C7290E94501864E670E080E0C9
:1032000090E00E94C7290115110551F32197E8CFDD
:10321000DF91CF911F910F910C945418809111352B
:1032200090911235A0911335B09114350196A11DDE
:10323000B11D8093113590931235A0931335B0933F
:10324000143540910401509105016091060170917F
:103250000701481759076A077B0710F510921135C7
:10326000109212351092133510921435609110356A
:1032700080910901861770F081E080930F3580916D
:103280000F35680F6093103570E08CE00E94662A5D
:103290000C945C1880910801681788F38FEFEDCFCC
:1032A00008958091113590911235A0911335B09108
:1032B00014350196A11DB11D8093113590931235DF
:1032C000A0931335B093143540910401509105013A
:1032D0006091060170910701481759076A077B073B
:1032E00010F510921135109212351092133510927C
:1032F00014356091103580910901861770F081E0D6
:1033000080930F3580910F35680F6093103570E012
:103310008DE00E94662A0C94541880910801681769
:1033200088F38FEFEDCF089560EC70E08BE499E3C4
:103330000E94491866E070E08BE499E30E94491806
:103340006091333970E08BE499E30E94491860EC96
:1033500070E08BE499E30C94491860EC70E08BE426
:1033600099E30E94491867E070E08BE499E30E94BA
:1033700049186091150170E08BE499E30E944918A7
:1033800060EC70E08BE499E30C94491860EC70E019
:103390008BE499E30E9449186FE070E08BE499E3B5
:1033A0000E94491861E070E08BE499E30E9449189B
:1033B00060EC70E08BE499E30C94491860EC70E0E9
:1033C0008BE499E30E9449186FE070E08BE499E385
:1033D0000E94491870E060E08BE499E30E9449186C
:1033E00060EC70E08BE499E30C94491860EC70E0B9
:1033F0008BE499E30E9449186EE070E08BE499E356
:103400000E9449188091313961E070E0811102C059
:1034100070E060E08BE499E30E94491860EC70E092
:103420008BE499E30C94491860EC70E08BE499E329
:103430000E94491868E070E08BE499E30E94491803
:1034400066E470E08BE499E30E94491860EC70E058
:103450008BE499E30C94491860EC70E08BE499E3F9
:103460000E94491860E570E08BE499E30E944918D6
:1034700061E070E08BE499E30E9449186EE170E02E
:103480008BE499E30E94491860EC70E08BE499E3C7
:103490000C94491860EC70E08BE499E30E944918A1
:1034A00068E470E08BE499E30E94491860E970E0F9
:1034B0008BE499E30E94491860EC70E08BE499E397
:1034C0000C94491860EC70E08BE499E30E94491871
:1034D00067E470E08BE499E30E94491861E370E0CF
:1034E0008BE499E30E94491860EC70E08BE499E367
:1034F0000C94491860EC70E08BE499E30E94491841
:1035000069E470E08BE499E30E94491861E970E096
:103510008BE499E30E94491860EC70E08BE499E336
:103520000C94491880913339882341F060913C39DB
:1035300070913D398AEA91E00C944A040895809193
:103540003339882341F060911801709119018AEA9A
:1035500091E00C942305089580932F39882321F05E
:1035600081E0809330390895109230390895809128
:103570003339882309F4E0C080912E39823A51F41E
:10358000609116017091170150E040E08AEA91E0E5
:103590000E94350380912E39833A51F460911601CF
:1035A0007091170150E040E08AEA91E00E943503F3
:1035B00080912E39843A51F460911601709117016F
:1035C00050E040E08AEA91E00E94350380912E3974
:1035D000873A51F4609116017091170141E050E073
:1035E0008AEA91E00E94350380912E39883A51F49D
:1035F000609116017091170141E050E08AEA91E074
:103600000E94350380912E39893A51F46091160158
:103610007091170141E050E08AEA91E00E94350381
:1036200080912E39833B51F46091160170911701FE
:1036300041E050E08AEA91E00E94350380912E3902
:10364000843B51F4609116017091170141E050E004
:103650008AEA91E00E94350380912E39883B51F42B
:10366000609116017091170141E050E08AEA91E003
:103670000E94350380912E39893B51F460911601E7
:103680007091170141E050E08AEA91E00E94350311
:1036900080912E39843C51F460911601709117018C
:1036A00041E050E08AEA91E00E94350380912E3992
:1036B000893C51F4609116017091170141E050E08E
:1036C0008AEA91E00E94350380912E39843E51F4BC
:1036D000609116017091170141E050E08AEA91E093
:1036E0000E94350380912E39893E51F46091160174
:1036F0007091170141E050E08AEA91E00E943503A1
:1037000080912E398E3F51F460911601709117010E
:1037100041E050E08AEA91E00E94350380912E3921
:103720008F3F51F4609116017091170150E040E015
:103730008AEA91E00C943503089580913339882307
:1037400061F08AEA91E00E940A026093383970932E
:10375000393980933A3990933B39089580913339C0
:10376000882371F0409138395091393960913A3954
:1037700070913B398AEA91E00E9489040C949D1B68
:10378000089580913339882361F08AEA91E00E949C
:10379000DA016093343970933539809336399093D8
:1037A0003739089580913339882371F04091343945
:1037B0005091353960913639709137398AEA91E004
:1037C0000E9458030C94C11B0895809133398823BB
:1037D00021F08AEA91E00C94280280E0089583EDBC
:1037E0009FE00E94471891E0833709F090E0892F0D
:1037F0000895C8E3DFE06FEFCE010E9433182196F1
:10380000C11580E1D807B9F70E94601888E39FE0EE
:103810000E944718982F81E0933021F0903F11F0DB
:1038200080E00895089589E39FE00E9447188093FF
:103830002E39843A49F0893A39F092E0980F81E0C4
:10384000923018F080E0089581E008958AE39FE0C7
:103850000E94471880932D399FEF980F81E09E3F7B
:1038600008F080E00895BF92CF92DF92EF92FF922E
:103870000F931F93CF93DF938BE090E00E94262855
:103880007C018C01C8E3DFE0CE010E944718F801FB
:1038900081938F012196C334FFE0DF07A9F76BE026
:1038A00070E0C7010E94FA17B82EC92E082F192FF1
:1038B000DD24D394CE010E944718F80191918F0125
:1038C0008913D12C2196C335FFE0DF0799F78B2DA3
:1038D0009C2D0E94C228C7010E94C2288D2DDF9115
:1038E000CF911F910F91FF90EF90DF90CF90BF90FD
:1038F00008958FED9FE00E94471891E0833709F00B
:1039000090E0892F0895CF92DF92EF92FF92CF93AC
:103910000E94791C882309F461C084ED9FE00E9415
:10392000471890E090933D3980933C3985ED9FE0B6
:103930000E94471890E0909319018093180186ED3A
:103940009FE00E94471890E0909317018093160122
:103950008BED9FE00E944718C82F8CED9FE00E94DE
:10396000471890E0B0E0A0E07C01DD24CC24FC2AE4
:103970008DED9FE00E944718C82F8EED9FE00E94BA
:103980004718C82ADC2AC0923439D0923539E092DF
:103990003639F092373987ED9FE00E944718C82FDB
:1039A00088ED9FE00E94471890E0B0E0A0E07C0125
:1039B000DD24CC24FC2A89ED9FE00E944718C82F03
:1039C0008AED9FE00E944718C82ADC2AC092383945
:1039D000D0923939E0923A39F0923B39CF91FF9049
:1039E000EF90DF90CF90089580913239882309F4C9
:1039F0008AC080913339882309F485C060913C39AD
:103A000084ED9FE00E9433186091180185ED9FE0DE
:103A10000E9433186091160186ED9FE00E943318D2
:103A2000609138397091393980913A3990913B39A8
:103A3000692F77278827992787ED9FE00E94331801
:103A4000609138397091393980913A3990913B3988
:103A5000BC018827992788ED9FE00E943318609168
:103A600038397091393980913A3990913B39672FC3
:103A7000782F892F992789ED9FE00E943318609154
:103A800038398AED9FE00E94331860913439709183
:103A900035398091363990913739692F77278827C2
:103AA00099278BED9FE00E94331860913439709113
:103AB00035398091363990913739BC01882799275B
:103AC0008CED9FE00E943318609134397091353944
:103AD0008091363990913739672F782F892F992720
:103AE0008DED9FE00E943318609134398EED9FE098
:103AF0000E94331863E78FED9FE00E9433188AE03D
:103B000090E00C94E6188AE090E00C94BA1860E01B
:103B10008FED9FE00C94331882E390E00E946F18C1
:103B20000E94F91B8091303970E060E0882319F021
:103B300060912F3970E08AEA91E00C9497058AEA47
:103B400091E00E9411031092333908958091343925
:103B500090913539A0913639B0913739892B8A2B1C
:103B60008B2BE1F08091383990913939A0913A3915
:103B7000B0913B39892B8A2B8B2B81F080911601D8
:103B8000909117018F3F910549F080913C399091B8
:103B90003D39892B19F010921501089581E0809329
:103BA000150108958091D101883C50F42091CF01F6
:103BB0003091D00181E02115384118F480E008955A
:103BC00081E00895CF938AEA91E00E944F01C82FC7
:103BD0000E94962960931A3570931B3580931C358B
:103BE00090931D35C0FF2DC081E0809325358093D3
:103BF00024358093233580911E3590911F35209177
:103C00002535211108C020912435211104C02091AF
:103C10002335222319F120910F01309110018217D1
:103C20009307B0F4019690931F3580931E3581E081
:103C300080932235809121358823E9F0CF910C942F
:103C40005018109225351092243510922335D3CF79
:103C500081E08093223580932135ECCF009741F0AD
:103C6000019790931F3580931E3510922235E2CF35
:103C700010922135FACFCF910C9454180F931F93C3
:103C80000E94962900911A3510911B3520911C3500
:103C900030911D35601B710B820B930B00910B0152
:103CA00010910C0120910D0130910E0160177107E8
:103CB0008207930720F01F910F910C94E21D1F9132
:103CC0000F9108951092900089E18093910080E80F
:103CD0009EE3909397008093960080E2809371001A
:103CE000089580910901809310350895803C61F416
:103CF0006BED70E08BE499E30E9449188CED682F1E
:103D00008BE499E30C940A2C8B3DC9F76BED70E0C2
:103D10008BE499E30E9449188DEDF1CF60EC70E0DF
:103D20008BE499E30E94491861E270E08BE499E327
:103D30000E94491880912D350E94761E80912C3565
:103D40000E94761E80912B350E94761E80912A3526
:103D50000E94761E60EC70E08BE499E30C944918A5
:103D600060EC70E08BE499E30E94491862E270E035
:103D70008BE499E30E944918809129350E94761EB0
:103D8000809128350E94761E809127350E94761EEC
:103D9000809126350E94761E60EC70E08BE499E3FA
:103DA0000C944918CF93C0911201C35660EC70E097
:103DB0008BE499E30E94491863E270E08BE499E395
:103DC0000E9449188C2F0E94761E60EC70E08BE4F4
:103DD00099E3CF910C94491860EC70E08BE499E37F
:103DE0000E94491864E270E08BE499E30E9449184C
:103DF00080912C390E94761E60EC70E08BE499E390
:103E00000C94491860EC70E08BE499E30E94491827
:103E100062E070E08BE499E30E94491880913B399D
:103E20000E94761E80913A390E94761E809139391F
:103E30000E94761E809138390E94761E60EC70E0F8
:103E40008BE499E30C94491860EC70E08BE499E3FF
:103E50000E94491861E070E08BE499E30E944918E0
:103E6000809137390E94761E809136390E94761EE5
:103E7000809135390E94761E809134390E94761ED9
:103E800060EC70E08BE499E30C944918CF93DF93D6
:103E9000C8E3DFE0CE010E9447180E94761E2196FB
:103EA000C11580E1D807B1F7DF91CF91089560EC9B
:103EB00070E08BE499E30E94491861E570E08BE4BF
:103EC00099E30E9449180E94461F60EC70E08BE461
:103ED00099E30C944918CF93C82F60EC70E08BE401
:103EE00099E30E94491860E970E08BE499E30E942D
:103EF00049186C2F8BE499E30E940A2C60EC70E067
:103F00008BE499E3CF910C944918CF93DF93C82F9A
:103F1000D62F0E94EF1B81110BC0C83C48F48C2F98
:103F200090E06D2F885C904FDF91CF910C94331807
:103F300083E0DF91CF910C946B1FCF93DF930E94AE
:103F4000A61DC0913339C11149C08091150181115D
:103F50003EC0D0913239DD23D1F1409134395091B6
:103F6000353960913639709137398AEA91E00E948B
:103F7000A703892B59F481E00E946B1F90E080E039
:103F80000E946F188C2FDF91CF91089581E080936C
:103F900033390E94B71A0E94AE1B0E94921A0E94E7
:103FA0009F1A0E94C11B8AEA91E00E94450568E9B8
:103FB00073E28AEA91E00E94A6020E94921D0E948A
:103FC000941983E090E00E94E618CD2FDBCF0E9489
:103FD000941983E090E00E94BA18D4CF0E949419FB
:103FE000D1CF60EC70E08BE499E30E94491864E063
:103FF00070E08BE499E30E94491860913C398BE4AE
:1040000099E30E940A2C60EC70E08BE499E30C9435
:10401000491860EC70E08BE499E30E94491865E070
:1040200070E08BE499E30E944918609118018BE4D9
:1040300099E30E940A2C60EC70E08BE499E30C9405
:10404000491860EC70E08BE499E30E94491869E03C
:1040500070E08BE499E30E94491860912F398BE45A
:1040600099E30E940A2C60EC70E08BE499E30C94D5
:10407000491860EC70E08BE499E30E94491863E012
:1040800070E08BE499E30E944918609116018BE47B
:1040900099E30E940A2C60EC70E08BE499E30C94A5
:1040A0004918CF93C82F60EC70E08BE499E30E942D
:1040B000491860E470E08BE499E30E9449186C2F82
:1040C0008BE499E30E940A2C60EC70E08BE499E3A6
:1040D000CF910C94491890911735992309F48EC209
:1040E000803C09F0ACC080910A0181119DC0109202
:1040F00017358091021D9091031D6091FE1C7091F7
:10410000FF1C8617970761F42091041D3091051D4F
:104110008091001D9091011D2817390709F471C283
:104120002091041D3091051D8091021D9091031D69
:1041300002972817390709F464C28091CF01909142
:10414000D0018115984108F05CC22091CB013091DB
:10415000CC018091CD019091CE01019710F48FEFA9
:1041600097E18217930709F44BC02817390708F025
:1041700042C0821B930B0196009709F442C2409102
:10418000D1014F5F4093D101E091041DF091051DD5
:10419000318320834091041D5091051D2091001D05
:1041A0003091011D4217530771F57093051D6093FF
:1041B000041DE0916A1BF0916B1B91838083209119
:1041C0006A1B30916B1B8091661B9091671B2817AF
:1041D000390721F58091641B9091651B90936B1BAF
:1041E00080936A1B8091CD019091CE019093CC0178
:1041F0008093CB010895821B930B8F5F974EBCCFAA
:1042000081E090E0BCCF2091041D3091051D2E5F10
:104210003F4F3093051D2093041DCBCF80916A1B27
:1042200090916B1B0296DACF81E0809317358EEF69
:1042300080930A0110921935109218350895209133
:104240001835309119352C3F91E0390708F0D9C164
:1042500090910A012115310529F49E3F19F48093AC
:104260000A010895911146C08B3D21F481E08093AD
:104270001635089590911635992349F08C3D21F01B
:104280008D3D19F48BED01C080EC109216359091A4
:10429000D101983C08F0B5C12091CF013091D001F7
:1042A0002115384108F0ADC12091CF013091D001E6
:1042B0002F5F3F4F3093D0012093CF012091CD014C
:1042C0003091CE01A9014F5F5F4F5093CE014093D3
:1042D000CD012E523E4FF90180838091CD01909106
:1042E000CE018115984109F08CC11092CE01109237
:1042F000CD010895913009F044C08B3DD1F49093E5
:1043000016358091183590911935049709F079C1C7
:1043100060912A3770912B3780912C3790912D37EF
:104320000E94672F6115710581059105D9F40C94E0
:10433000241F90911635992349F08C3D21F08D3D35
:1043400019F48BED01C080EC10921635A9014F5F76
:104350005F4F5093193540931835265D384CF9015D
:104360008083CFCF60933439709335398093363959
:1043700090933739809114018131C9F60E94D21B84
:10438000D6CF923009F045C08B3DD9F481E08093BF
:1043900016358091183590911935049709F031C17F
:1043A00060912A3770912B3780912C3790912D375F
:1043B0000E94672F6115710581059105D9F40C9450
:1043C000021F90911635992349F08C3D21F08D3DC7
:1043D00019F48BED01C080EC10921635A9014F5FE6
:1043E0005F4F5093193540931835265D384CF901CD
:1043F0008083CFCF609338397093393980933A39BD
:1044000090933B39809114018131C9F60E94AE1B13
:10441000D6CF933099F48F3F11F40C943920823128
:1044200008F081E190E0909317018093160180914C
:104430001401813191F70E94B71AEFCF9430D1F473
:104440008F3F11F40C94F11F863088F090E08D308E
:10445000910514F08CE090E090933D3980933C39C5
:1044600080911401813171F70E94921AEBCF86E09E
:1044700090E0F2CF9530D1F48F3F11F40C940920E5
:10448000853088F090E08930910514F088E090E064
:10449000909319018093180180911401813171F773
:1044A0000E949F1AEBCF85E090E0F2CF993021F483
:1044B0000E94AC1A0C942120963079F48F3F11F4AD
:1044C0000C949419811103C00E949F1DF9CF813073
:1044D00009F097C00E949D1FF3CF913211F40C9404
:1044E0008E1E923211F40C94B01E933211F40C947F
:1044F000D21E973021F40E94A61D0C94AD19903362
:1045000019F490E00C94E618903421F40E94E51B15
:104510000C945120983029F4833709F072C00C9420
:10452000141A9E3059F4813021F4809331390C945F
:10453000F6198111FCCF10923139F9CF9F3041F437
:104540000E94D21D811102C00C94C6190C94DE1970
:10455000993529F4883F09F054C00E948C1D953587
:1045600029F4883F09F04DC00E946018913511F47C
:104570000C94571F923551F58B3D79F481E080936F
:10458000163580911835909119350297D1F56091C3
:104590002B3780912A370C94851F909116359923DB
:1045A00049F08C3D21F08D3D19F48BED01C080EC7C
:1045B00010921635A9014F5F5F4F50931935409304
:1045C0001835265D384CF9018083DBCF903511F426
:1045D0000C942C1A983411F40C944A1A993411F44E
:1045E0000C947A1A973411F40C94621A933511F4DE
:1045F0000C94F41C943529F40C94871D803C09F428
:1046000013CE089581E08093C8014FB7F8942091AC
:104610000B3530910C3580910D3590910E354FBF93
:1046200028173907F1F0E0910B35F0910C358091A6
:10463000093590910A35E817F90761F4809107353B
:104640009091083590930C3580930B3580810E94B2
:104650006B20DBCFE0910B35F0910C35CF0101964B
:10466000F1CF1092C8010895CF93DF9360EC70E012
:104670008BE499E30E94491870E060E08BE499E3D1
:104680000E944918CEE2D7E320912A3930912B3984
:10469000CE018E52974382179307C8F46991603C0C
:1046A00061F46BED70E08BE499E30E9449186CEDC6
:1046B0008BE499E30E940A2CE7CF6B3DC9F76BEDC1
:1046C00070E08BE499E30E9449186DEDF1CF60EC46
:1046D00070E08BE499E30E94491810922B391092F4
:1046E0002A39DF91CF910895CF93DF93EC01209782
:1046F000E1F0219780912A3990912B398C3F91409C
:10470000A0F48AEA91E00E94BF0120912A393091F9
:104710002B39A9014F5F5F4F50932B3940932A39B2
:10472000225D384CF9018083E2CFDF91CF9108956B
:104730000F931F93CF93DF93EC0180913139811157
:104740007BC08AEA91E00E94BF012197409111014C
:1047500080FF57C09C0154E0359527955A95E1F7A5
:104760002F7033274F3FD9F410922B3910922A39EA
:10477000209311018AEA91E00E946601909313014F
:10478000809312018AEA91E00E94520180932C39B1
:10479000CE01DF91CF911F910F910C9474232413BC
:1047A000E3CF8AEA91E00E946601209112013091E4
:1047B0001301820F931F97FD01969595879590930E
:1047C00013018093120100912C3910E08AEA91E0E4
:1047D0000E945201800F912F911D9595879580938E
:1047E0002C39CE010E9474238FEF809311010E9417
:1047F000D21E0E94EC1EDF91CF911F910F910C945D
:1048000034234F3F39F010922B3910922A398FEF11
:10481000809311018AEA91E00E946601909313014E
:10482000809312018AEA91E00E94520180932C3910
:10483000CE010E947423DBCF10922B3910922A39BB
:10484000E9CFCF92DF92EF92FF920F931F93CF9316
:10485000DF93EC0180913339882309F479C080918A
:104860003139811153C00E94581860E071E080E036
:1048700090E00E94852D162F107FCF3FD10508F0C4
:10488000116070E060E08AEA91E00E947605612F95
:104890008AEA91E00E94B1009EE2C92E95E3D92EEA
:1048A000C25DDA4CEE24E394F12CCC16DD06F1F077
:1048B000F60161916F018AEA91E00E94B100FFEF79
:1048C000EF1AFF0A8FEFE816F10479F78AEA91E010
:1048D0000E942B0270E060E08AEA91E00E94760577
:1048E000612F8AEA91E00E94B100DCCF8AEA91E070
:1048F0000E942B020E945C18DF91CF911F910F91B3
:10490000FF90EF90DF90CF900C94921D0E9458186A
:10491000CF3FD10519F010F0CFEFD0E080913039C2
:1049200070E060E08111BE018AEA91E00E947605A4
:104930000EE215E3C8018E5295438C179D07B0F621
:10494000F80161918F018AEA91E00E94B100F2CFF3
:1049500082E00E946B1F85E090E0DF91CF911F9174
:104960000F91FF90EF90DF90CF900C946F180F9302
:104970001F93CF93DF938091C90181116EC081E0B5
:104980008093C901C0E0D8E14FB7F8942091021D8F
:104990003091031D8091041D9091051D4FBF281774
:1049A000390709F45AC0E091021DF091031D80916E
:1049B000001D9091011DE817F90709F03FC0809193
:1049C000FE1C9091FF1C9093031D8093021D00819B
:1049D0001181E091681BF091691B2091661B309159
:1049E000671BE217F30789F52091641B3091651B63
:1049F0003093691B2093681B20813181A9014150AC
:104A000051094C3F514008F0BFCFEEE2F5E30E52A2
:104A10001543C8018E0F9F1FBE010E94092FDC01A4
:104A2000AE52BE4F8C918193CF018E529543821727
:104A3000930778F3C9010E942124A6CFE091021DBB
:104A4000F091031DCF010296BECFE091681BF0915B
:104A5000691B9F012E5F3F4FCBCF1092D101109267
:104A6000D0011092CF011092C901DF91CF911F9117
:104A70000F910895809133398823E1F10E943E1E01
:104A80008091D101882311F180912035811102C0DC
:104A90000E94E21D80912235811128C0809121352C
:104AA000811124C080912035882331F062E370E0C9
:104AB00080E090E00E94C7290E94E21D809122358B
:104AC000811104C0109220350E94B7244FB7F8948A
:104AD00020910B3530910C3580910D3590910E352C
:104AE0004FBF2817390791F00C94022381E080937F
:104AF0002035ECCF80913239882319F00E940E19AD
:104B0000E5CF0E9451190E949F1DE0CF0895CF93D9
:104B10008091CA01811127C081E08093CA01C4E15C
:104B20008BE499E30E94802B892BD9F08FB7F894FE
:104B300040910B3550910C35209107353091083557
:104B40004217530791F440910D3550910E35209145
:104B5000093530910A354217530739F48FBFC150D8
:104B6000F9F61092CA01CF91089540910D355091F8
:104B70000E3520910B3530910C35215031094217FB
:104B8000530761F38FBF8BE499E30E949A2B2FB7F1
:104B9000F894E0910D35F0910E35808340910D35FC
:104BA00050910E358091093590910A354817590773
:104BB00051F4809107359091083590930E3580938C
:104BC0000D352FBFCCCF80910D3590910E350196CC
:104BD000F4CF1F920F920FB60F9211240BB60F92C3
:104BE0002F933F934F935F936F937F938F939F93F5
:104BF000AF93BF93EF93FF930E948725FF91EF91AF
:104C0000BF91AF919F918F917F916F915F914F91E4
:104C10003F912F910F900BBE0F900FBE0F901F90E2
:104C200018958091EC3980FF2AC082E08093153579
:104C30008091153581508230B8F50E94EF1B882392
:104C400081F10E94061C882361F10E94131C8823B5
:104C500041F10E94261C882321F10E94331C8823E5
:104C600051F181E0809332390E94791C882319F137
:104C70000E94831C82E1809314010C949D1F82FF8B
:104C800002C083E0D3CF83FF02C081E0CFCF42E2F6
:104C900050E065E571E08BE499E30E944A2D0E94A3
:104CA000A518109232390895109232394EE150E031
:104CB00068E771E0F0CF089580E00E94482A0E94E2
:104CC0007D2DA6E0BDE181E098E1FD019C011192FE
:104CD00021503040E1F7E7E0F5E3B183A083B783EB
:104CE000A683B583A48386E095E39383828326E03D
:104CF00040E052EC61E070E08BE499E30E94512CBB
:104D00000E94621E61E08CE00E94162B61E08DE043
:104D10000E94162BEEE2F7E38CEF91E0DF019C019D
:104D20001D9221503040E1F7EAE2F7E384E0DF0131
:104D30001D928A95E9F7E2EDF1E080E098E1DF016C
:104D40009C011D9221503040E1F7ACE6BBE182E9C5
:104D500091E0FD019C01119221503040E1F7EEEF0E
:104D6000FCE1B183A083B783A683B583A4832CEF32
:104D70003CE133832283A2EDB9E1FD019C01119254
:104D800021503040E1F7E4E6FBE1B183A083B78333
:104D9000A683B583A48382E69BE19383828322E08A
:104DA00030E043E050E064E070E08AEA91E00E9485
:104DB000F7000C941126CF93CFB7F8948091413926
:104DC000811127C0E0EDF0E08491E0EBF0E09491F8
:104DD000E82FF0E0EE0FFF1FEA50FF4FA591B491CE
:104DE000EC91E92321F461E084E00E94522B61E020
:104DF00084E00E94162B8CB580618CBD8CB58064DC
:104E00008CBD61E087E00E94162B61E085E00E9486
:104E1000162B809141398F5F80934139CFBFCF915D
:104E200008959FB7F89480914139882319F08150F3
:104E30008093413980914139811105C08CB58F7BB8
:104E40008CBD109240399FBF08952FB7F8948130E0
:104E500041F0C0F08230A1F082E08093403980E0E0
:104E600001C082E090913F39892B80933F39809136
:104E70004039811103C081E0809340392FBF0895EC
:104E800084E0F0CF81E0EECF909140399230A1F0F4
:104E90009FB7F894833088F4E82FF0E0E956FE4F8E
:104EA0008081809520913F39822380933F39811101
:104EB00002C0109240399FBF089580E0F2CF08955C
:104EC000833060F5E82FF0E0EE0FFF1FE65EFE4F47
:104ED00071836083813051F08230A1F0809169004C
:104EE0008C7F482B40936900E89A0895809169006F
:104EF000837F440F551F440F551F482B4093690073
:104F0000E99A0895809169008F7C94E0440F551FC1
:104F10009A95E1F7482B40936900EA9A0895833007
:104F200078F4E82FF0E0813061F0823061F0E898A9
:104F3000EE0FFF1FE65EFE4F8FE597E291838083C1
:104F40000895E998F5CFEA98F3CF1F920F920FB624
:104F50000F9211240BB60F922F933F934F935F93B1
:104F60006F937F938F939F93AF93BF93EF93FF9331
:104F7000E0911A01F0911B010995FF91EF91BF910A
:104F8000AF919F918F917F916F915F914F913F91E1
:104F90002F910F900BBE0F900FBE0F901F90189582
:104FA0001F920F920FB60F9211240BB60F922F93F0
:104FB0003F934F935F936F937F938F939F93AF93A1
:104FC000BF93EF93FF93E0911C01F0911D010995B0
:104FD000FF91EF91BF91AF919F918F917F916F91D1
:104FE0005F914F913F912F910F900BBE0F900FBE8D
:104FF0000F901F9018951F920F920FB60F921124C9
:105000000BB60F922F933F934F935F936F937F93C2
:105010008F939F93AF93BF93EF93FF93E0911E0104
:10502000F0911F010995FF91EF91BF91AF919F9171
:105030008F917F916F915F914F913F912F910F9041
:105040000BBE0F900FBE0F901F9018950F931F93DC
:10505000CF93DF938230910510F482E090E0E091ED
:10506000EA39F091EB3930E020E0B0E0A0E0309791
:1050700099F42115310509F44AC0281B390B243055
:105080003105D8F58A819B816115710589F1FB0194
:1050900093838283FE0111C040815181028113817B
:1050A00048175907E0F04817590799F4109761F02D
:1050B00012960C93129713961C933296CF01DF91A0
:1050C000CF911F910F9108950093EA391093EB3916
:1050D000F4CF2115310551F04217530738F0A901DB
:1050E000DB019A01BD01DF01F801C1CFEF01F9CF6A
:1050F0009093EB398093EA39CDCFFE01E20FF31F95
:10510000819391932250310939832883D7CF2091FD
:10511000E8393091E939232B41F420912201309173
:1051200023013093E9392093E8392091200130910F
:1051300021012115310541F42DB73EB740912401DD
:1051400050912501241B350BE091E839F091E939A4
:10515000E217F307A0F42E1B3F0B2817390778F04E
:10516000AC014E5F5F4F2417350748F04E0F5F1FAD
:105170005093E9394093E839819391939FCFF0E0C0
:10518000E0E09CCFCF93DF930097E9F0FC013297EA
:1051900013821282A091EA39B091EB39ED0130E02F
:1051A00020E01097A1F420813181820F931F20917C
:1051B000E8393091E9392817390709F061C0F093CF
:1051C000E939E093E839DF91CF910895EA01CE17EC
:1051D000DF07E8F54A815B819E0141155105B1F772
:1051E000E901FB83EA8349915991C40FD51FEC175C
:1051F000FD0761F4808191810296840F951FE9017A
:1052000099838883828193819B838A83F0E0E0E0A5
:1052100012968D919C9113970097B9F52D913C9121
:105220001197CD010296820F931F2091E83930919A
:10523000E9392817390739F6309751F51092EB39CB
:105240001092EA39B093E939A093E839BCCFD383FF
:10525000C28340815181840F951FC817D90761F41B
:105260004E5F5F4F88819981480F591F518340835A
:105270008A819B81938382832115310509F0B0CF08
:10528000F093EB39E093EA399ECFFD01DC01C0CF0A
:1052900013821282D7CF08951F920F920FB60F92EA
:1052A00011242F933F938F939F93AF93BF9380913C
:1052B000433990914439A0914539B09146393091A4
:1052C000423923E0230F2D3758F50196A11DB11D5A
:1052D000209342398093433990934439A0934539C0
:1052E000B09346398091473990914839A091493916
:1052F000B0914A390196A11DB11D80934739909311
:105300004839A0934939B0934A39BF91AF919F91E1
:105310008F913F912F910F900FBE0F901F90189576
:1053200026E8230F0296A11DB11DD2CF2FB7F89406
:105330006091433970914439809145399091463953
:105340002FBF08953FB7F89480914739909148391D
:10535000A0914939B0914A3926B5A89B05C02F3F85
:1053600019F00196A11DB11D3FBFBA2FA92F982F8B
:105370008827BC01CD01620F711D811D911D42E086
:10538000660F771F881F991F4A95D1F708958F924E
:105390009F92AF92BF92CF92DF92EF92FF926B01FA
:1053A0007C010E94A2294B015C01C114D104E104DB
:1053B000F104E9F00E944B290E94A2296819790999
:1053C0008A099B09683E73408105910570F321E0CD
:1053D000C21AD108E108F10888EE880E83E0981E11
:1053E000A11CB11CC114D104E104F10429F7FF9000
:1053F000EF90DF90CF90BF90AF909F908F900895E7
:10540000789484B5826084BD84B5816084BD85B59F
:10541000826085BD85B5816085BDEEE6F0E0808166
:1054200081608083E1E8F0E0108280818260808387
:10543000808181608083E0E8F0E08081816080830A
:10544000E1EBF0E0808184608083E0EBF0E080813C
:1054500081608083E1E9F0E08081826080838081E7
:1054600081608083E0E9F0E0808181608083EAE709
:10547000F0E080818460808380818260808380818D
:10548000816080838081806880831092C10008954C
:10549000883020F0873108F487E188512091260177
:1054A00090E4299F900111248770822B80937C00C7
:1054B00080917A00806480937A0080917A0086FDE2
:1054C000FCCF809178009091790008951F93CF933D
:1054D000DF93182FEB0161E00E94162B209739F41F
:1054E00060E0812FDF91CF911F910C94522BCF3F21
:1054F000D10511F461E0F5CFE12FF0E0E457FF4F63
:10550000E491E150EA3008F054C0F0E0E657F54D80
:105510000C945E2F942A9C2AA12AAB2AD92AD92A34
:10552000B52ABD2AC52ACF2A84B5806884BDC7BDE7
:10553000DF91CF911F91089584B5806284BDC8BD6D
:10554000F7CF80918000806880938000D09389009D
:10555000C0938800EDCF80918000806280938000AE
:10556000D0938B00C0938A00E3CF8091B000806815
:105570008093B000C093B300DBCF8091B000806215
:105580008093B000C093B400D3CF80919000806826
:1055900080939000D0939900C0939800C9CF8091D8
:1055A0009000806280939000D0939B00C0939A00FB
:1055B000BFCFC038D1050CF09DCF92CF81508A303B
:1055C00080F5E82FF0E0E951F54D0C945E2FFB2AB1
:1055D000FF2AF12AF72A112B112B022B082B0C2B57
:1055E000122B809180008F778093800008958091A6
:1055F00080008F7DF9CF84B58F7784BD089584B501
:105600008F7DFBCF8091B0008F778093B00008959D
:105610008091B0008F7DF9CF809190008F7780933B
:1056200090000895809190008F7DF9CFCF93DF9304
:1056300090E0FC01E455FF4F249184539F4FFC01FF
:1056400084918823C9F090E0880F991FFC01EA50EB
:10565000FF4FA591B491FC01E451FF4FC591D49146
:1056600061110DC09FB7F8948C91209582238C9383
:105670008881282328839FBFDF91CF9108956230CE
:1056800051F49FB7F8943C91822F809583238C939B
:10569000E8812E2BEFCF8FB7F894EC912E2B2C9323
:1056A0008FBFEACF1F93CF93DF93282F30E0F9010C
:1056B000E457FF4F8491F901E455FF4FD491F9016C
:1056C000E453FF4FC491CC23A9F0162F81110E94FF
:1056D000DE2AEC2FF0E0EE0FFF1FE451FF4FA59103
:1056E000B4918FB7F894EC91111108C0D095DE23D6
:1056F000DC938FBFDF91CF911F910895DE2BF8CF00
:10570000FC01918D228D892F90E0805C9F4F821B40
:1057100091098F7399270895FC01918D828D9817B7
:1057200031F0828DE80FF11D858D90E008958FEFA7
:105730009FEF0895FC01918D828D981761F0A28DE5
:10574000AE0FBF2FB11D5D968C91928D9F5F9F73A1
:10575000928F90E008958FEF9FEF089583E19DE28F
:10576000892B49F080E090E0892B29F00E94132DCD
:1057700081110E94000080E090E0892B49F080E0D8
:1057800090E0892B29F00E94000081110C94000008
:105790000895FC01A48DA80FB92FB11DA35ABF4FC6
:1057A0002C91848D90E001968F739927848FA68920
:1057B000B7892C93A089B1898C9180648C93938D47
:1057C000848D981306C00288F389E02D80818F7D37
:1057D00080830895CF93DF93EC01888D8823B9F0FF
:1057E000AA89BB89E889F9898C9185FD03C08081EC
:1057F00086FD0DC00FB607FCF7CF8C9185FFF2CF69
:10580000808185FFEDCFCE010E94C92BE9CFDF91CA
:10581000CF910895EF92FF920F931F93CF93DF9351
:10582000EC0181E0888F9B8D8C8D981316C0E889E0
:10583000F989808185FF11C0EE89FF896083E8893D
:10584000F98980818064808381E090E0DF91CF914D
:105850001F910F91FF90EF900895F62E0B8D10E0A1
:105860000F5F1F4F0F731127E02E8C8D8E110CC010
:105870000FB607FCFACFE889F989808185FFF5CF5B
:10588000CE010E94C92BF1CFEB8DEC0FFD2FF11D46
:10589000E35AFF4FF0820B8FEA89FB898081806297
:1058A000D2CFCF92DF92EF92FF921F93CF93DF93ED
:1058B000EC016A017B01122FE889F98982E080837B
:1058C000C11481EED806E104F104A1F060E079E0B2
:1058D0008DE390E0A70196010E941D2F2150310910
:1058E000410951095695479537952795211580E12E
:1058F000380798F0E889F989108260E874E88EE149
:1059000090E0A70196010E941D2F21503109410905
:1059100051095695479537952795EC85FD85308338
:10592000EE85FF852083188EEC89FD891083EA8936
:10593000FB89808180618083EA89FB89808188601E
:105940008083EA89FB89808180688083EA89FB897A
:1059500080818F7D8083DF91CF911F91FF90EF90A9
:10596000DF90CF9008951F920F920FB60F921124DF
:105970000BB60F922F938F939F93EF93FF93E0912A
:105980005B39F0915C398081E0916139F091623945
:1059900082FD1DC09081809164398F5F8F7320914B
:1059A0006539821741F0E0916439F0E0E55BF64C2F
:1059B000958F80936439FF91EF919F918F912F91F3
:1059C0000F900BBE0F900FBE0F901F901895808107
:1059D000F2CF1F920F920FB60F9211240BB60F92B7
:1059E0002F933F934F935F936F937F938F939F93E7
:1059F000AF93BF93EF93FF938BE499E30E94C92B7E
:105A0000FF91EF91BF91AF919F918F917F916F9196
:105A10005F914F913F912F910F900BBE0F900FBE52
:105A20000F901F9018958BE499E30E94802B21E042
:105A3000892B09F420E0822F0895EBE4F9E3138227
:105A4000128288EE93E0A0E0B0E084839583A68381
:105A5000B7838EE991E09183808385EC90E0958710
:105A6000848784EC90E09787868780EC90E0918B28
:105A7000808B81EC90E0938B828B82EC90E0958B15
:105A8000848B86EC90E0978B868B118E128E138E12
:105A9000148E0895AF92BF92CF92DF92EF92FF9251
:105AA0000F931F93CF93DF936C017B018B01040F46
:105AB000151FEB015E01AE18BF08C017D10759F0E2
:105AC0006991D601ED91FC910190F081E02DC60124
:105AD0000995892B79F7C501DF91CF911F910F911E
:105AE000FF90EF90DF90CF90BF90AF900895FC01B2
:105AF00044835583668377830895009729F0BC011A
:105B000090E080E00C94EC300895CF92DF92EF9219
:105B1000FF926B017C01C114D104E104F10441F056
:105B20000E949D30A70196010E943F2F6B017C01CE
:105B3000C701B601FF90EF90DF90CF9008950895D0
:105B40000E94002A0E949F2D0E945C26CEEADBE282
:105B50000E943A252097E1F30E94AE2BF9CF0E94D4
:105B6000272E08F481E008950E94BB2D6894B1119E
:105B70000C94962E08950E947B2E88F09F5798F0E3
:105B8000B92F9927B751B0F0E1F0660F771F881F42
:105B9000991F1AF0BA95C9F714C0B13091F00E945C
:105BA000952EB1E008950C94952E672F782F8827B5
:105BB000B85F39F0B93FCCF3869577956795B39583
:105BC000D9F73EF490958095709561957F4F8F4FF2
:105BD0009F4F0895E89409C097FB3EF490958095F7
:105BE000709561957F4F8F4F9F4F9923A9F0F92FA3
:105BF00096E9BB279395F695879577956795B79521
:105C0000F111F8CFFAF4BB0F11F460FF1BC06F5F06
:105C10007F4F8F4F9F4F16C0882311F096E911C018
:105C2000772321F09EE8872F762F05C0662371F039
:105C300096E8862F70E060E02AF09A95660F771F4D
:105C4000881FDAF7880F9695879597F90895990F29
:105C50000008550FAA0BE0E8FEEF16161706E80736
:105C6000F907C0F012161306E407F50798F0621B57
:105C7000730B840B950B39F40A2661F0232B242B2C
:105C8000252B21F408950A2609F4A140A6958FEF4B
:105C9000811D811D089597F99F6780E870E060E09D
:105CA00008959FEF80EC089500240A9416161706B5
:105CB00018060906089500240A94121613061406FD
:105CC00005060895092E0394000C11F4882352F060
:105CD000BB0F40F4BF2B11F460FF04C06F5F7F4F18
:105CE0008F4F9F4F089557FD9058440F551F59F0FF
:105CF0005F3F71F04795880F97FB991F61F09F3FB9
:105D000079F087950895121613061406551FF2CFE1
:105D10004695F1DF08C0161617061806991FF1CF31
:105D200086957105610508940895E894BB27662758
:105D30007727CB0197F908950E94AF2E0C94622E1D
:105D40000E94542E38F00E945B2E20F0952311F013
:105D50000C944B2E0C94512E11240C94962E0E94D0
:105D6000732E70F3959FC1F3950F50E0551F629FFE
:105D7000F001729FBB27F00DB11D639FAA27F00DA4
:105D8000B11DAA1F649F6627B00DA11D661F829FCB
:105D90002227B00DA11D621F739FB00DA11D621FB0
:105DA000839FA00D611D221F749F3327A00D611DCD
:105DB000231F849F600D211D822F762F6A2F1124AF
:105DC0009F5750409AF0F1F088234AF0EE0FFF1FE2
:105DD000BB1F661F771F881F91505040A9F79E3F39
:105DE000510580F00C944B2E0C94962E5F3FE4F3FB
:105DF000983ED4F3869577956795B795F795E7958F
:105E00009F5FC1F7FE2B880F911D9695879597F997
:105E10000895AA1BBB1B51E107C0AA1FBB1FA617F1
:105E2000B70710F0A61BB70B881F991F5A95A9F743
:105E300080959095BC01CD010895A1E21A2EAA1B70
:105E4000BB1BFD010DC0AA1FBB1FEE1FFF1FA2172A
:105E5000B307E407F50720F0A21BB30BE40BF50B27
:105E6000661F771F881F991F1A9469F760957095B0
:105E7000809590959B01AC01BD01CF010895052E41
:105E800097FB1EF400940E94562F57FD07D00E94E6
:105E90001D2F07FC03D04EF40C94562F50954095BF
:105EA000309521953F4F4F4F5F4F089590958095C6
:105EB000709561957F4F8F4F9F4F0895EE0FFF1F95
:105EC0000024001C0BBE0790F691E02D0994692771
:105ED0009627692778278727782708950E943930E1
:105EE000A59F900DB49F900DA49F800D911D11242E
:105EF0000895E894DF93CF93FC01DB010E943930D1
:105F00007F936F93E9019A01AC01BF93AF933F93E5
:105F10002F93DF010E94393026F46C1B7D0B820B1E
:105F2000930B9E01EB01FC010E944830AF91BF91A1
:105F30002F913F910E944830BE01CF01F9012F916E
:105F40003F91CF91DF910895689401C0E8948F92BA
:105F50009F92CF93DF930E94B22FDF91CF919F90BA
:105F60008F90089588249924F401E401B0E49F936C
:105F7000AA279A158B049C04ED05FE05CF05D007D2
:105F8000A10798F4AD2FDC2FCF2FFE2FE92D982CF1
:105F9000892E982F872F762F652F542F432F322F3E
:105FA0002227B85031F7BF9127C01B2EBF91BB27C6
:105FB000220F331F441F551F661F771F881F991F0D
:105FC000881C991CEE1FFF1FCC1FDD1FAA1FBB1FC3
:105FD0008A149B04EC05FD05CE05DF05A007B1077B
:105FE00048F08A189B08EC09FD09CE09DF09A00BCF
:105FF000B10B21601A94E1F62EF49401AF01BE01B9
:10600000CD01000C0895002E083090F0982F872FB6
:10601000762F652F542F432F322F22270850F4CF8D
:10602000220F331F441F551F661F771F881F991F9C
:106030000A95B2F7002D089597FD1094002E0830B0
:1060400098F00850232F342F452F562F672F782F85
:10605000892F912DF4CF159497958795779567950E
:1060600057954795379527950A95AAF71124002D3E
:106070000895A29FB001B39FC001A39F700D811D21
:106080001124911DB29F700D811D1124911D089541
:106090000E943930460F571FC81FD91F08F4319688
:1060A00008958F929F92AF92BF92CF92DF92EF921C
:1060B000FF92CF93DF93EC01688179818A819B8184
:1060C000611571058105910521F464E279ED8BE597
:1060D00097E02DE133EF41E050E00E943F2F49016E
:1060E0005A019B01AC01A7EAB1E40E946E2F6B013B
:1060F0007C01ACEEB4EFA50194010E941E31C60EE6
:10610000D71EE81EF91EF7FE06C081E0C81AD108A6
:10611000E10880E8F80AC882D982EA82FB82C701D6
:10612000B6019F77DF91CF91FF90EF90DF90CF90F6
:10613000BF90AF909F908F9008958F929F92AF9253
:10614000BF92CF92DF92EF92FF9260910001709127
:106150000101809102019091030161157105810592
:10616000910521F464E279ED8BE597E02DE133EFC1
:1061700041E050E00E943F2F49015A019B01AC01D0
:10618000A7EAB1E40E946E2F6B017C01ACEEB4EF84
:10619000A50194010E941E31C60ED71EE81EF91EED
:1061A000F7FE06C081E0C81AD108E10880E8F80AC5
:1061B000C0920001D0920101E0920201F09203012D
:1061C000C701B6019F77FF90EF90DF90CF90BF900F
:1061D000AF909F908F90089560930001709301019C
:1061E00080930201909303010895FB01DC0102C03A
:1061F00001900D9241505040D8F70895DC0101C044
:106200006D9341505040E0F70895F999FECF92BD4B
:1062100081BDF89A992780B50895262FF999FECF68
:106220001FBA92BD81BD20BD0FB6F894FA9AF99AB3
:106230000FBE01960895B7FF0C946E2F0E946E2F2B
:0A624000821B930B0895F894FFCF22
:10624A0001000000F82A00002801FE030000000FE8
:10625A0000FFDCFE1101FF0005005F275F275F27B3
:10626A000000ED39800001781E00A02800F03C00F3
:10627A00405100127A00E4A20024F40048E8019098
:10628A00D00320A10700000000B1004502B101BF00
:10629A00018002C7004572726F722C20696E6465B4
:1062AA007465726D696E61746520626F6F742076B1
:1062BA006563746F720D0A004572726F722C2069E1
:1062CA006E636F727265637420626F6F7420766595
:1062DA0063746F720D0A00010204000000000A2CA8
:0A62EA004A2D802B9A2B8C2BEA2BF7
:00000001FF
